:020000040000FA
:040000000CD003D04D
:08000800FFD0550EA76EAA0EF1
:08001000A76EA6820000120099
:08001800F5D0A66A0F0EA96ED7
:10002000A680A848EDD010EE00F0D96AF36AF46A11
:10003000F482CB0E926E80688168C90E936E4F0E6B
:10004000826E949C948E900EAB6E260EAC6E829A4D
:10005000949A82989498AB98030ED56EACD8ABD88E
:10006000810EAF6EAE50AE50AE50AB88AB98AB8841
:100070009AD80F0AE6E100EE08F0006A016A93D808
:100080000F0AF6E00450040A0AE00450050A01E1F0
:100090008AD804500026EE6E014ED3D7F0D7005216
:1000A000D0E10A50F66EA96E0B50F76E0CC0F8FF47
:1000B00000EE0DF00950016ED8B4FF00085004089E
:1000C000C0E3FA6AFB6A0844F926BBD703D00ED016
:1000D0001FD033D00900F5CFEEFF012EFBD7020E63
:1000E000F424E8AEAED70950050F33D0F80EF6165B
:1000F000080EEECFF5FF0D00E82EFBD70A00840EA8
:10010000A66E83DF0900012EF1D7F7CFD9FF20D0EB
:10011000940EA66E7ADFF350F61807E1F450F71844
:1001200004E1400EF326E86AF422400EF626E86A5F
:10013000F722F822012EECD70BD0A66AA680A8CF12
:10014000EEFFA94AA92A012EF8D70950050F01D0C0
:10015000010E828A828810EE00F0016E0F0E1FD809
:100160001ED8006A00EE08F0EE5000260CD8012ED2
:10017000FBD7006C005007D8040E11D8ACA2FED7F4
:10018000829A82985ED7056E0F0A06E00550040A2F
:1001900003E00550050A02E1050E01D805509EA8AE
:1001A000FED7AD6E1200ABB2FF0004009EAAFDD7D1
:1001B000AE50046E1200D76AD66AD58E809AF2A429
:1001C00012D0F294020EF46203D0E2B219D004D03D
:1001D000D9AC02D0E1B414D0E4508086809AE1B664
:1001E0008096E1B6808A040082BEE9D7808A808644
:0C01F000040082AEFDD7D59E1200004630
:10020000E2EF03F0E2EF03F0D8CF3CF03E6E9E50F9
:100210009D14300B03E1F2A403D0F2BAA5EC18F060
:10022000F2A20BD08290CEEC11F0F292F2883F0E47
:10023000306E070E2FEC10F082809E509D14300B14
:1002400003E1F2A403D0F2BAA5EC18F09EB056EC8C
:1002500004F03E503CC0D8FF1000005F010EF76E66
:10026000F668F86A000E0A00F524F7AEFCD7E866D7
:100270003D807D0EF76EBF0EF66E000EF86A0A0026
:10028000F524F7AEFCD7E8663D8005EEEFF0AA0E48
:10029000EFCF39F0EF6EEF623D82EF42EF12EF3EAB
:1002A0003D8239C0EDFFEAA6F3D7A69EA69CA96AB7
:1002B000000EA680A818A92AFCE1E828FE0B82906F
:1002C000306A010E2FEC10F0AA0E306E020E2FECE9
:1002D00010F0301E020E2FEC10F0040E1DEC10F08A
:1002E0007F0B020AE8663D8A020E1DEC10F0AA0A96
:1002F000E8663D8A020E1DEC10F0550AE8663D8A5C
:10030000010E1DEC10F03F0BE8663D8A040E1DEC5B
:1003100010F07F0BE8663D8A3F0E306E070E2FEC23
:1003200010F0306A2B0E2FEC10F00A0E306E2A0EF1
:100330002FEC10F0306AC00EF0EC11F0010E21EC41
:1003400002F0070E1DEC10F0E8BA3D8C010E21EC16
:1003500002F0070E1DEC10F0E8AA3D8C81B03D8C38
:100360003F0E306E070E2FEC10F081A03D8C3DBC8F
:100370003D8A8280F66AF76A829A82BE04D00900BA
:10038000F7A6FBD73D860F0EA96EFF0EB1EC0BF062
:10039000020E21EC02F051A00AD0D0A608D0D180E4
:1003A000FF0E21EC02F0FF0E21EC02F03D8E810EDB
:1003B000C26EC284010EF46E23EC02F0C2B43D881A
:1003C000C4503D5001E1120095683DBA956AAA0EED
:1003D000836E080E306E3DA0819A3DB08198280E44
:1003E000831E841E21EC02F00400818A8188280E7D
:1003F000831E841E21EC02F004003D42302EEBD718
:10040000809A0A0E21EC02F0808A0A0E21EC02F09A
:10041000819A0A0E21EC02F0818A0A0E21EC02F088
:1004200080960A0E21EC02F080860A0E21EC02F082
:1004300081980A0E21EC02F081880A0E21EC02F06C
:100440001200F46AF48EF36AF32EFED7F42EFCD772
:10045000E82CF7D71200810EC26E4E0EC16EC10E8F
:10046000926E80688168C10E936E4F0E826E800E10
:10047000946E836A070EB46E000E956E846A000E49
:10048000966E000C020ED56E810ECD6EB10EB16E61
:10049000180ECB6E010EBE6E200EBD6E9494040E2F
:1004A000CA6E2C0EBD6E000C05EEFFF0ED6AE95031
:1004B000FDE1EA50FBE1EF6A000CAC98AC849C0EC5
:1004C000396402D0FF0E21D04E0E396402D0810E65
:1004D0001CD02C0E396402D0400E17D01E0E396489
:1004E00002D02A0E12D0150E396402D0200E0DD083
:1004F0000F0E396402D0150E08D00B0E396402D0ED
:100500000F0E03D0090E396E0A0EAF6E396E640EEF
:10051000AC6EB00EAB6E000CF29E3968F76AF66AEC
:10052000000EF468F368D968E96810EE00F082BE46
:100530002ED0E65282AEFDD7E250F76204D0E150F1
:10054000F664F66E05D0F760FDD7E1CFF6FFF76EE3
:10055000020E82AE13D0E8481ED082BEFCD73960AE
:10056000396E3950070DF450F7620AD0F350F66037
:10057000000C10EE03F082AEDCD709D00000F1D7FA
:10058000F760000C10EE03F082AED3D700D082AE3D
:1005900013D0E83CFCD782AE0FD0E92EF8D782AE5C
:1005A0000BD00400D92EF3D739503E60000C51B067
:1005B000FF0C393C000CFF0C3948BBD7D2D7330EA7
:1005C000E96201D0340C350EE96201D0300C370EEF
:1005D000E96201D0350C3F0EE96201D0320C390ED0
:1005E000E96201D0330CE950300AF00B02E1E95026
:1005F0001200EAB20ED0E9B63F0CE950070BE9B899
:10060000E886E9BAE888E9BCE88AE9BEE88C400FE8
:100610001200C00EE9603F0C700EE9241200DFECFE
:1006200002F0A96E350EA91832E137AC23D0379C01
:10063000350EA96E000EABEC0BF0310EA96E010E5B
:10064000316EABEC0BF0300EA96E1F0E356FABECBC
:100650000BF0330EA96E810E356FABEC0BF0400E34
:10066000A96EFF0EABEC0BF0A92A300EA962F9D7E8
:10067000378C000C040E37B408D037A8179037A871
:1006800003D001A217800190FF0EE92A01D0EE509D
:10069000E92AE84805D0E804ABEC0BF0E866120064
:1006A00036063650BCE1000CE86620D0310ECAECAC
:1006B00008F0E84804D0E80402E0E8AE316E330EFA
:1006C000CAEC08F0E84802D0E804396E320ECAECF1
:1006D00008F0E84802D0E8043F6E350ECAEC08F096
:1006E000E84804D0E804376E3794371A300ECAEC65
:1006F00008F0E84802D0E804356E340ECAEC08F081
:10070000E84804D0E804F00F100FD8B06009336E49
:100710000F0BBE6E1200800EF16E000EF06E000E1A
:100720009E6E000EA16E000EA46E210E9D6E000E38
:10073000A06E000EA36E000E9F6E000EA26E000E45
:10074000A56E000ED06ED00EF26ED180000C360E6B
:10075000CAEC08F0E83C120003EEF0F0B2CFEFFF75
:10076000010E366E360EA96E12EC03F0B3CFEFFF1A
:10077000010E366E370EA96E12EC03F01200B40EA5
:10078000F66E070E03D0A40EF66E070EF76EF86A2B
:1007900011EE50F0100E306E0900F550E66E302E5E
:1007A000FBD71200C107000800000000000003F0A2
:1007B00008000C02C17000100000000000000200E0
:1007C00008000C022BEC02F054EC02F05180F42CE7
:1007D00003D0F32C01D0519042EC02F082909DECBA
:1007E00010F082802EEC01F08096809AA69EA69C46
:1007F000010E316E600E336E000EBE6E358835828E
:100800003580358435863F82000E54EC03F0395034
:1008100051823F8C3F8A3F883E6E8CEC02F0E8BEEE
:100820000CD0518003EEF0F039C0EFFF010E366EB0
:10083000330EA96E12EC03F005D051903E50D8B49F
:10084000640E396E5DEC02F03DEC16F0310E3B6E3D
:10085000A7EC03F00F0EA96E010E3D14FF0ED8A4F5
:10086000FE0EB1EC0BF0020E21EC02F00182C3ECA3
:1008700003F03468000082909EEC1BF082803DEC17
:1008800016F08BEC03F07CEF0FF09D989D9AF29A96
:10089000AB9E82883FBE05D0D8B0828CD8A0829C07
:1008A0001200D8B0829CD8A0828C12009E90320692
:1008B000808A8086818A81883FA619D017A204D0B9
:1008C000D88001A0D8900DD017AA0DD020EEE1F06D
:1008D000DD2E06D0DF6603D0D890179A02D0DF064F
:1008E000D88045EC04F082BC809A120008D051B642
:1008F00080963FA402D082AE809651B4809A01B215
:1009000006D001A036D025668198819A120001AAEE
:1009100030D03B48120038BE04D0C00E386E3A6A60
:1009200012003BC0D9FFDA6A0F0ED9BEDA6E3A2A3E
:100930003ABA382A3A9AC10E381803E1DAA6DF6AC1
:10094000389C38A41200819ADF66818A819838A089
:1009500003D0800E381612003A661200DF2ADF98A4
:10096000F00E3316BE500F0B331231661200312ACF
:10097000120038BE386A3A2A3ABC382A3A9C38986B
:100980003BC0D9FFDA6A0F0ED9BEDA6E3828DF60B5
:1009900004D031661200312A12003C0E3A64120073
:0409A000819A120026
:10100000000EE3502DEC08F0E8BC000C06D0000EFA
:10101000E3502DEC08F0E8AC000C0E0EE3AC000C35
:101020003FA4000C010EE3CF42F0429E020EE830D6
:10103000D8B002D04236FBE3D89042320B0EE3CF59
:10104000E9FF0A0EE3CFEAFFEE50EDCFEEFFEE6EC2
:10105000422EFAD70E0EE39C010C1E0A03E1BE0ECF
:101060003B6E100C040A03E1310E3B6E100CBB0A00
:1010700001E1100C600A01E1400C010A01E1000CE1
:10108000C00A01E1000CE20A01E1200C280A01E19A
:10109000200C070A01E1200C270A01E1200C070AB5
:1010A00001E1200C3B68C90A01E1800C010A01E161
:1010B000800C030A01E1800C010A01E1800C000CA4
:1010C00034502DEC08F0D8A4000CE8A81200310E22
:1010D000CAEC08F0311809E0010E366E310EA96E27
:1010E000310EE96EEA6A12EC03F0340ECAEC08F035
:1010F0000F0BBE18D8B41200010E366E340EA96E56
:10110000BE0EE96E0F0EEA6EF00E3316EF500F0BA7
:10111000331212EC03F0120060EC08F034502DECA6
:1011200008F0D8A4000CE8AE010CF29EBFEC03F06E
:10113000F28E010C000EE350426E020EE3CF2BF054
:10114000030EE3CF2CF0010EE3CF1DF01D9E020E27
:10115000E830D8B0000C2C362B36D8B0020C1D3637
:10116000F7E3030CEE50D90A14E1EE50380A11E10E
:10117000EE505C0A0EE1EE505D0A0BE1EE50D10A32
:1011800008E1EE50E00A05E1EE505C0A02E1EE50A3
:10119000A10A1200A96EA680A85012004244366E21
:1011A000DFEC02F03F0A05E13F0AA96EEF50ABEC1D
:1011B0000BF0EE50362EF4D74244E95E1200F00EEA
:1011C000E1160E0EE3AE37D00B0EE3CF5EF0090E44
:1011D000E350426E0F0B366E362A42380F0B426ECA
:1011E000365E366C010EE350E89E5D6A5D2A362459
:1011F00002E0FCE21FD0010E5DC0E3FFD8905D3637
:10120000D88031504254426EF29E5D02F46611D095
:10121000F350F28E366E5E260B0EE35036260B0E22
:1012200036C0E3FFD8805E504266000E5E5A5D26EF
:1012300002D0F28E030C030ED890E334E96E020E56
:10124000E334EA6EF00B379E07E0020EE350FE0B2C
:10125000E00AD8A4020C378E010EE350E89E426EDD
:10126000000EE3502DEC08F0D8A4030CE834E83469
:101270000B0EE3CF36F00A0EE3CFE2FF36C0E1FFFC
:10128000D8A0A0D037BE020C060EE260020C010E00
:10129000E218D8B4020C000EE2B411D0E2A208D0D9
:1012A000E00EE114D8B4020C000EE2B0180E07D024
:1012B0005F0EE164020CE00EE86CE830E89E422428
:1012C000D8B0030CE834D8B0030CE804E124D8B05B
:1012D000030C0F0EEA1804E0EA50FC0BE866020C5F
:1012E0004250D890E834D8B0030CE804E92404E371
:1012F000030EEA60030C07D0EAA605D0600BD8A461
:1013000033D0E9AE030C020EEA621FD01F0EE9646F
:101310001CD0220EE96207D020C0E6FF03C0E6FF22
:1013200002EE20F012D0200EE9620BD000C0E6FFE2
:1013300001C0E6FF20C0E6FF03C0E6FF02EE20F09A
:1013400004D0E906E906E906E906EA6606D0300EA9
:10135000E918F00B02E1E66AE94AEECFE6FFEECFCC
:10136000E6FF422EF2D7000CFE0EE962020C0F0ED1
:10137000EA62020C010E4262030CF29EF86A590EF8
:10138000F66E2E0EF76E0900F550E8BC090FE8382E
:10139000F00B426E09000900F550E8BC090F0F0B75
:1013A0004210E66E0900F550E8BC090FE838F00B72
:1013B000426E0900F550F28EE8BC090F0F0B421087
:1013C000E66E000CEA50FC0BE866020C4250D89026
:1013D000E834D8B0030CE804E924D8B0030CEAA23E
:1013E0000FD0300FD8B0020C1F0EE964020CBAEC1B
:1013F0000AF037AE000CEAA0020CCEEC08F0000CAC
:10140000EAA011D05F0EE964020C206ABAEC0AF07F
:1014100043EC0BF0E848030C42C036F0360637BE0A
:10142000CEEC08F0000CC70FD8B093D02F0EE964B3
:1014300074D0366A310EE96013D03650E3501F0A7B
:10144000DF0BD8A4030C3628E350000AD8B4030CF1
:101450000F0AF00BD8A4030CB5EC0AF03EE003D061
:10146000330EE9600BD03650E3500F0A03E0FF0A59
:1014700001E0030C3628B5EC0AF02FE0350EE960E8
:1014800012D03650E350446E441E1F0A04E01F0A77
:101490005F0BD8A4030C3628E3504414D8A4030CE3
:1014A000B5EC0AF01AE03650E350446E441E010ACF
:1014B0000BE0030A09E0060A07E0140A05E0300A17
:1014C00003E0600A01E0030C3628E3504414D8A47A
:1014D000030CB5EC0AF001E0030C366AE9CFA9FF72
:1014E000E92A3650E350446E441CEF163628E35088
:1014F0004414EE12330E010FE91803E133500F0BC1
:10150000BE6EB5EC0AF0ECE1A928E96E37B801929D
:1015100042C036F00FEC03F0000C040EE9620BD071
:10152000040E326E248E32BE04D024BEFCD701B02D
:10153000000C249E040C020EE962020C010E4262B1
:10154000030CE766030C010EE366030C026A036AF0
:10155000000CDF0EE964020C4250D890E834DF0F33
:10156000D8B0030CBAEC0AF0000C362A362A364002
:101570004218120042C036F0E6CFEEFFE6CFEEFF93
:10158000422EFAD73650426EE95EE95EE15EE15ED8
:10159000000CA69EA69CA96A12EE00F0A680A85098
:1015A000E66EA92AE166FAD7000EE8A009D012EE8D
:1015B00000F0E1CFA9FFE650ABEC0BF0E166F9D704
:1015C00012EE00F0310EE34804D0E80402E0E8AE89
:1015D000316E330EE34802D0E82C396E320EE34808
:1015E00002D0E82C3F6E350EE34804D0E804376E95
:1015F0003794371A300EE34802D0E82C356E340E9B
:10160000E34808D0E804F00F100FD8B06009336E3B
:101610000F0BBE6E400EE16E0A0E426E01EE58F0E8
:10162000080EE926E6CFEEFFE82CFCD7422EF8D7CD
:1016300043EC0BF0900EE16E020EE26E700E03EEC4
:1016400020F0E6CFEEFFE82CFCD7E16A020EE26E56
:10165000300EE6CFEEFFE82CFCD71200E350B10AC3
:10166000D890E8300EE1010EE344E89008E3442608
:10167000D8B0FF0CCF0E4464FF0CD880FF0C362688
:10168000FF0CD890000C429E010EE26E600EE16EDF
:10169000200E446E200E366E0A0E44C0E3FF000E8C
:1016A000E35045E02DEC08F0D8A43ED0200A0EE12E
:1016B000000EE3500F0B0D0A04E0020E2EEC0BF0AF
:1016C00033E2040E2EEC0BF02FE218D0000EE330C4
:1016D000010EE3BE29D0E3AC04D0E39CE36624D042
:1016E000E38CE344FE0B20E003E336261DE206D044
:1016F00044261AE2CF0E446401D016D00C0EE36AE1
:10170000E3820D0EE36A0F0EE36AE3820E0EE390AE
:10171000E382E384E386E398E39A100EE126BCE3D8
:1017200042AE000C429EFF0C000EE368428E0E0E8D
:10173000E396E394E392E39AF0D703EE60F0A69E7B
:10174000A69C000EA96E600EA680A8CFEEFFA92A67
:10175000E804FAE11200426E0F0EA918D8B4020C88
:101760004250426EA86E020E326EA684F29E550E54
:10177000A76EAA0EA76EA682F28E32BE02D0A6B2C5
:10178000FCD7A694A6804250A862030C000C0E0E53
:10179000E3AE08D0365006E0E36A0F0EE36A519AD2
:1017A0005198000C0D0E36C0E3FF0F0EE36AE38480
:1017B000500EE16412000D0EE36601D0100CE350F0
:1017C000040A120017AE30D000B40CD012EE00F0B4
:1017D000E76A12EE04F0E76A12EE08F0E76A12EE2A
:1017E0000CF0E76A206A032AD8B0022A026624981D
:1017F000200EE16E010EE26E179E37A602D017840E
:1018000013D017940E0EE3A60BD0E3A209D0E38405
:101810000F0EE36AE3820C0EE39EE39CE39AE398E7
:10182000100EE126EEE3010C415021E0E16E010EC5
:10183000E26E0F0EE350040A1AE10E0EE3A60CD07E
:10184000E3A40AD0E3A208D0DBEC0BF0E86604D0F6
:101850000F0EE36AE382040C416A37A804D001B298
:10186000040C1780019001A207EC08F0040C405012
:101870004AE0E16E010EE26E0F0EE350020A43E110
:1018800000EC08F088EC0CF0E8B22DD0E8B422D0DF
:10189000040E01B202D001B013D017900E0EE3B0C7
:1018A0000CD037A815D001B213D0100E326E01B093
:1018B00007D032AEFCD717800BD001B224D0000C79
:1018C0000E0EE3BE07D0E384415001E0000C020C91
:1018D000040E01D0020E366E4050E16E010EE26E33
:1018E000C7EC0BF0000C37A802D001A21780DFEC88
:1018F00008F0366E4050E16E010EE26E07EC08F023
:10190000C7EC0BF0000CA0EC0CF0E866080C000C27
:10191000020EE350E00BA00A0EE1020EE3341E0BB0
:10192000D8B4020C00EEE0F0E926020EEECFE3FFA1
:10193000030EEFCFE3FF020EE350E8AE010C020C02
:101940003FB604D037B602D001A0000C415009E0E8
:10195000E16E010EE26E0F0EE304FE0B020A01E1DE
:10196000000C200E01B230D0E16E010EE26E446A2E
:10197000426A0E0EE350E8BA06D0E8A40BD00F0E70
:10198000E350020A07E10C0EE350426003D0E1CFBE
:1019900044F0426E100EE12637B407D037B205D0BE
:1019A00037B003D0600EE16005D0000EE222020ED7
:1019B000E262DFD7425003E137903796000C44C013
:1019C000E1FF010EE26E010C500E446E010E12009A
:1019D000C10E01EE50F0446E000E44C0EBFF010E4C
:1019E000E3CFEBFFEB9E0E0EEB6AEB86EB840F0E64
:1019F000EB6AEB841200446EE3CF36F0020E36C081
:101A0000EBFF4428E3CF36F0030E36C0EBFF020EA7
:101A1000EB50B00A0DE1810E366E020E36C0EBFFC0
:101A20000A0EE330E88E366E030E36C0EBFF000C74
:101A3000020EEB50366E200FD8B0000C400FD8A02D
:101A40001DD00F0BD8B4020CE84400EEE0F0E926FC
:101A500036BC0DD0EECF36F0EFCF42F001EE50F0B5
:101A6000020E36C0EBFF030E42C0EBFF000C36A89F
:101A7000020CEACF36F0E9CF42F0F0D7070EEBCFF9
:101A800036F0030EEB503626030E36C0EBFF060E83
:101A9000EBCF36F0020EEB503622020E36C0EBFFD3
:101AA000000C446EE350E00BA00AD8A41AD000EE5C
:101AB000E0F04450E3343E0BE8BA04D0E926442871
:101AC000E35009D0E89AFE0FD8A0000C020FE926D7
:101AD000010EE350E89EEC26D8A0000CE906EF2AA0
:101AE000000CC00AD8B4000C040E4462000C01EED5
:101AF00050F0010EE3CF44F0070EEB504422070EE6
:101B000044C0EBFF446A060EEB504422060E44C06C
:101B1000EBFF000CE1CF42F00E0EE3A60BD0E3A2E8
:101B200009D0E3840F0EE36AE3840C0EE39EE39C8A
:101B3000E39AE398100EE124E16E4462EDD742C0CF
:101B4000E1FF1200500EE164000C0C0EE350100F88
:101B5000446E0C0E44C0E3FF090EE3504418D8B4A1
:101B60000000F00E4414100A64E1600EE11807E171
:101B700000EEE2F0810EEE6E100EEE6E378601EE94
:101B800050F00D0EEB6AE36A060EEB6A070EEB6A85
:101B9000060EE350C00F06E3040EEB6A050EEB6A77
:101BA000EB8012D0040EEB660FD0050EEB660CD066
:101BB000060EE3CF44F0040E44C0EBFF070EE3CF64
:101BC00044F0050E44C0EBFF0C0EE388E39AE39C5F
:101BD000000EE3502DEC08F0E8AA27D0000EE350E9
:101BE0000F0B0D0A0EE1010EE3CF44F000EE60F0A2
:101BF000020EE3CFEEFF030EE3CFEEFF442EF8D745
:101C000014D0E8EC0CF00D0EEB6A600E446E0B0E77
:101C100044C0EBFF0A0EEB6A020EFBEC0CF0020E66
:101C200051EC0DF011EE50F0000C0C0EE39CE3981B
:101C3000E38A01EE50F0060EE350C00B0EE0060EF4
:101C4000E3A60BD0E3500F0B0D0A07E10D0EEBB22C
:101C5000E382EBB4E384EB6A03D00D0EEB662ED186
:101C60000C0EE350F00B200AD8A453D0E8EC0CF093
:101C7000000EE3502DEC08F0E8BA34D0040EEB6A05
:101C8000050EEB6AEB80000EE3CFEBFF020EE3CF15
:101C9000EBFF030EE3CFEBFF0C0EE398E39AE38C2C
:101CA000E1CF44F0000EE330030ED8B0020E426ED6
:101CB0000A0E42C0EBFFE3CF42F00B0E42C0EBFF37
:101CC0000EE310EEE3F0E734E890426E0B0E42C0F4
:101CD000EBFF010EEB50E89EE526D8B0E72A11EEA7
:101CE00050F0000C01EE50F0000EE350F00BC00A73
:101CF0000DE0A00E446E0B0E44C0EBFF0A0EEB6A23
:101D0000040EFBEC0CF011EE50F0000C0C0EE3880E
:101D100003D0100A01E04CD0000EE350F00BC00AD3
:101D20003668D8A4366A00EE60F0020E426EEFCF3D
:101D300044F0400EEB503666000E441A07E042A213
:101D400005D04292EF64428042A04284400E36A009
:101D500044C0EBFFE92A5F0EE95C446E010EE344E8
:101D6000E8904464E4D701EE50F0090E42C0EBFF66
:101D7000060EE350C00F02E3E8AA15D0C00EE9EC4E
:101D80000CF0A00E3666600E446E0B0E44C0EBFFE6
:101D90000A0EEB6A040EFBEC0CF0040E51EC0DF095
:101DA00011EE50F0000C040E51EC0DF001EE50F06D
:101DB000000EE3502DEC08F0E8AA75D0060EE350B3
:101DC000C00FD8A070D001EE50F0090EEBCF42F05A
:101DD000060EE350E8A613D0426A0F0B0D0A04E189
:101DE0000D0EE3660CD00AD0060A03E101A007D06D
:101DF00005D0010A04E117A402D017944286060E0A
:101E0000E350E8AC08D0421606E1070EE3500F0B92
:101E1000060A22E1FF0E42161792070EE3503F9E7C
:101E2000E8B63F8E070B18E0070A03E1179A1782FE
:101E300013D0020A0EE0030A06E1FF0E422451B25B
:101E400045EC04F007D000EEE0F0060AEF6E01EE7C
:101E500050F0178A51B23F86060EE350E8AE02D02A
:101E6000425021E020D0070EE350F00B1CE0500F51
:101E700007E3E8AC04D0446A8AEC0DF014D013D028
:101E8000E16004D0446E8AEC0DF00DD0E1CF42F059
:101E9000E16E01EC0CF042C0E1FF01EE50F00F0EDC
:101EA000EB6AEB8202D001EE50F0050EEB2E8CD6E1
:101EB000040EEB5003E0040EEB0686D601EE50F064
:101EC0000C0EE39EE39CE39AE398E150B00F206E82
:101ED0000D0EEB5003E00F0B201203D0010EE3AE0A
:101EE00003D0446A8AEC0DF0040EEB6A050EEB6A2F
:101EF0000F0EEBCFE3FFFF0C00C0E0F101C0E1F1FA
:101F000002C0E2F103C0E3F1E2EC0BF0E850F4E0D0
:101F100001A243D0E8B403D0E8B2EED73ED00F0E12
:101F2000E36AE3820D0EE35006E0019A070EE32A0E
:101F3000E3B225D0E1D703EEF0F0B2EC08F01FE1F8
:101F4000070EE36AEF50018A346213D0030EE350A8
:101F5000F00B23E00D0EE35002E0346A05D034505C
:101F6000D5EC0AF034B20BD0F29EC3EC03F0F28E43
:101F700014D0346E8CEC08F00009D8A40ED060ECBC
:101F800008F0019A0192310E3B6E24880F0EE36A2D
:101F900037A4B2D7C9EC0AF0AFD7A0EC0CF0E850E8
:101FA000ABE044C0E1FF010EE26EA2EC0DF0E8668A
:101FB000A3D703EEFFF0E1CFEFFF88EC0CF0E8B021
:101FC00010D0E8A20ED0DFEC08F0366E03EEFFF082
:101FD000EFCFE1FF010EE26E07EC08F0C7EC0BF06B
:101FE0008BD70F0E416AE36AE380E3829AEC08F034
:101FF000E85006E001D0030E366EC7EC0BF07CD73C
:1020000042502DEC08F01788E8AC17982496E8BAEF
:0C20100004D0E150F00B416E6FD7EDD70B
:022020000000BE
:0E20220022EE00F0000E306E30501DEC10F07B
:10203000DE6E302A30ACF9D71200956A8D6EE84416
:10204000E838070B8009836E8D50846A82968286F9
:102050008D6E956882920000835082821200956A8C
:102060008D6EE844E838070B8009836E8D50846AD2
:10207000829682868D6E3050956A836E82968286B5
:102080001200956A810E836E846A82968286010EA2
:10209000846E95688292000083508282080B956A54
:1020A0000109836E82968286846A800E836E829690
:1020B0008286010E846E836A82968286020E846E08
:1020C0001200956A810E836E846A82968286010E62
:1020D0008D6E95688292000083508282F70B956A1C
:1020E000836E82968286120035BC120001B2120005
:1020F000956A830E836E846A82968286842A9568A6
:102100008292000083508282FC0B301001B00309E0
:10211000956A836E82968286120035BC120001B2E7
:102120001200956A820E836E846A82968286848209
:102130003050836E8296828612008084F468F32E7B
:10214000FED7F42EFCD78094F468F32EFED7F42E3D
:10215000FCD7F468F32EFED7010E1DEC10F0E8500A
:1021600002E0F42EF7D7800E306E000E2FEC10F048
:10217000010E1DEC10F0020E306E3A0E2FEC10F036
:10218000F40E306E3D0E2FEC10F0030E306E2D0E5F
:102190002FEC10F0800E156E13EEE0F0E668E668A6
:1021A000E668E668E668E66800EE80F013EEE0F0C8
:1021B00017EC11F013EEE0F0B00EE66EE828E66ED4
:1021C000E828E66EE828E66EE828E66EE828E66E7F
:1021D00000EE8CF013EEE0F017EC11F013EEE0F0EF
:1021E000F80EE66E400EE66E100EE66EB10EE66E6E
:1021F000CC0EE66E000EE66E00EE98F013EEE0F008
:1022000017EC11F013EEE0F0A00EE66EE828E66E93
:10221000E828E66EE828E66EE828E66EE828E66E2E
:1022200000EEA4F013EEE0F017EC11F0120041EC18
:1022300010F0E950836E82968286EA50836E829611
:102240008286060E236EE750F00B306EE8383010B1
:10225000F00A836E82968286E6500F0B306EE83865
:102260003010F00A836E82968286232EECD7010E00
:10227000306E010E2FEC10F0EE50EAB805D0050ECE
:102280001DEC10F0E8ACF8D7306A010E2FEC10F01E
:10229000000C956A231C836E82968286221C836EB4
:1022A00082968286956A840E846A836E829682867E
:1022B000020E846E30C083FF82968286800E846A0E
:1022C000836E82968286010E846E1A0ED8B01E0E20
:1022D000836E82968286000CB80ED890303202E36C
:1022E000301AD890303202E3301AD890303202E3FC
:1022F000301AD890303202E3301AD890303202E3EC
:10230000301AD890303202E3301AD890303202E3DB
:10231000301AD890303201E3301A30501200956AEA
:10232000836E82968286231A2338F00B2318F46E6C
:10233000E8380F0B2218236ED890226AF434223624
:10234000E8342236E8342236231AF450221A1200D6
:10235000956A836A838E8384846A8296828630C07B
:1023600083FF8484829682868406836E8296828628
:102370001200F86A0B0E1C6E846A956A0A000B0044
:10238000F550836E82968286842A0B00F550836E08
:1023900082968286842A1C2EF2D7000C0500266ABB
:1023A0002250FE6E2350FD6EFF6A956A800E836E8A
:1023B000846A82968286070E8D6E956882920000EE
:1023C00083CF30F08282956A3F0E836E829682863A
:1023D000305012002686FECF22F0FDCF23F00600FB
:1023E000956A836A838E83808384846A82968286D8
:1023F000836E040E846E82968286810E836E846A5A
:1024000082968286010E846E9568829200008350C7
:102410008282080B956A0209836E82968286800EFC
:10242000836E846A82968286060E846E2650A00988
:10243000836E82968286BF0A836E8296828612009F
:10244000956A306EE86ADFCF83FFDE188296828657
:102450003006F9E11200956AD890E828E830D8A053
:1024600008D0DECF83FF82968286DECF83FF8296FE
:102470008286DECF83FF82968286DECF83FF8296BE
:102480008286E804EEE11200306EDE508FEC11F02F
:102490003006FBE1120016501F02F350306E956AB1
:1024A000800E836E846A82968286020E8D6E956897
:1024B0008292000083508282DE62000C302EF8D7B8
:1024C000010C040F306E956A800E836E846A8296CA
:1024D0008286020E8D6E9568010E17B829288282B9
:1024E0008292E82CFCD783508282D890303204E369
:1024F000D890303208E20FD0303209E230068292B2
:10250000DE6E835082828292DE6E8350828282925D
:10251000DE6E835082828292DE6E83508282302E03
:10252000EED7DE6E010C20EE0CF0DE6ADE6ADE6AAB
:10253000DE6ADE6ADE6ADE6ADE6A080E20EE04F01B
:10254000306E179C956A800E836E846A82968286AE
:10255000020E8D6E95688292000083508282DF6247
:10256000178CDE6E302EF7D71200306E41C0D9FFC7
:10257000010EDA6E0F0EDB6ADB840D0E30C0DBFF5E
:10258000120001B01200306E4150D8B41200D96E62
:10259000010EDA6E0F0EDB50030AD8A412000F0EE4
:1025A000DB6ADB840D0E30C0DBFF120041C0D9FFB7
:1025B000010EDA6E0A0EDBCF2DF00B0EDBCF2EF004
:1025C000120080824150809208E0D96E010EDA6ECE
:1025D0000F0EDB50030A01E101A0000C010CFC0E00
:1025E0001C6482D01C3C34D02B501A6204D02C5076
:1025F0001B64020C02D01A64020C1D042C24306EE1
:10260000000E2B201A6204D030501B64030C02D041
:102610001A64030C16042C14296E1650E83003E2D9
:102620002B322C32FBD717B8A4D016C01EF029527B
:1026300009E0E00E2E6E030E2D6E1786010E1F6E42
:102640001C06FF0C1F6A1DC01CF0D6EC12F04CD00B
:10265000D6EC12F01CB024D0E1CF23F0E2CF22F070
:102660002DC0E2FF2EC0E1FF23EEE0F01604306E35
:102670002950D92601E3DA2AE81CE82830141D6421
:102680001D50E6CFDEFFE82CFCD717961C0623C0B2
:10269000E1FF22C0E2FFE00E2E6E030E2D6EFF0C56
:1026A0001DC01CF01604306E2950E81CE8283014B8
:1026B0001C6484D01C5E2E26000E2D222C2A2B2278
:1026C0001C5016640BD010D01F502C2601E32B2A6F
:1026D0001602F3502E2601E32D2A1C5E18501C60B2
:1026E00035D016501C603AD017B85DD01C50166417
:1026F000EBD73DE0E00E2E6222D0030E2D6221D0FA
:10270000E1CF23F0E2CF22F0D6EC12F01C501D5C9A
:102710002E26000E2D222DC0E2FF2EC0E1FF23EE5B
:10272000E0F0E6CFDEFF1C2EFCD7179623C0E1FFBA
:1027300022C0E2FFE00E2E6E030E2D6EFF0C2E6EF9
:10274000030E2D6E010E1F6E1786FF0C1F6E1650A6
:1027500001D01F32E830FDE31796FF0C1CC01FF0BC
:10276000165001D01F32E830FDE31796FF0C1F6AA8
:10277000000C1DC01CF0D6EC12F0178629501C244A
:10278000196005E319501F6E2950195C02D01F6EA5
:102790001C501E6E1C5E16041F26165001D01F32E0
:1027A000E830FDE3FF0C296A1E502E26000E2D2274
:1027B0001F502C26000E2B221C66DFD71C6A1F6AB6
:1027C000000C824B3F032F3F3F00838B14C068E017
:1027D0000100840828FFFF0035A0CDD100B002D051
:1027E00001B0C9D101A02A6AC20EF66E270EF76E9B
:1027F000B9EC11F03338030B306E74EC10F0030EAB
:10280000EBEC11F001A009D001B407D001BE05D056
:102810005B0E306E110E2FEC10F041EC10F0260E16
:10282000836E82968286010E836E82968286000E69
:1028300024BE400E2A6E01B0400E836E82968286C0
:10284000E8500AE0E2CFDAFFE1CFD9FF24AE20EE74
:1028500004F0080E20EC12F02C0E306ED88052ECF2
:1028600011F02688400EEBEC11F030BA6FD1070E54
:10287000EBEC11F0030E1DEC10F0700A700BE86623
:1028800065D1360EEAEC11F030BA60D10A0E1DECBB
:1028900010F03F0BE8665AD1020E1DEC10F000005C
:1028A000020E1DEC10F0000093EC12F0256A01B44A
:1028B00009D01B6A010E1A6E300E196E040E186EC6
:1028C000166E01802A66249E00803338030B306E1A
:1028D00074EC10F017BC178E230E011620EE0AF0D0
:1028E000080EDF6211D0018ED906DFB209D0166E54
:1028F000186E100E196E070E1A6ED00E1B6E3BD09E
:102900001A6AE80E1B6E37D0040EDF620DD01A6A09
:10291000010E1A6EFE0E09A200001B6E040E196E47
:10292000186E040E166E27D0160EDF6207D00188CF
:10293000200E1B6E080E186E166E1DD00186050E39
:10294000DF1805E10196018C040E1A6E14D0020EF8
:10295000DF1811E1019601840ED0F00E0914080A67
:102960000AE0020A08E01A6A196A1B8C19841A0A1A
:1029700002E01B9C1B8600C0E0F101C0E1F102C037
:10298000E2F103C0E3F105C0E4F104C0E5F107C0E2
:10299000E6F106C0E7F109C0E8F108C0E9F10BC0B3
:1029A000EAF10AC0EBF1E1EC12F0E82CE4D01C688B
:1029B000256A050EEBEC11F0EFEC12F0E8BE09D041
:1029C000B5EC12F03066D7D0020EEBEC11F004003B
:1029D000D2D717B648D041EC10F0220E01B6620EE5
:1029E000836E82968286210E836E8296828620EE88
:1029F00004F0080E20EC12F02C5001B80D0F836E7D
:102A0000829682862EC0D9FF2DC0DAFF165020ECA8
:102A100012F02C0E306ED88001B6D89052EC11F026
:102A200026882684640EEBEC11F030BA78D001A62B
:102A300004D0900EEBEC11F016D001BCFAD7FC0ECE
:102A4000EAEC11F030BA6BD00A0E1DEC10F03F0B1F
:102A500001E065D0020E1DEC10F0E8B060D0050E6C
:102A6000EBEC11F0A9D741EC10F0220E836E8296A8
:102A70008286FE0E1B18200E03E001B41A67230E97
:102A8000836E8296828620EE04F0080E20EC12F00F
:102A90002C5001B80D0F836E829682861F04836EC0
:102AA000FE0E1B1804E001B41A67829682862C0E73
:102AB000306ED88052EC11F02688460EEBEC11F007
:102AC00030BA2DD00B0EEBEC11F0030E1DEC10F014
:102AD000700B700AE86623D0D50EEAEC11F030BA1C
:102AE0001ED00A0E1DEC10F03F0B01E018D0020EB4
:102AF0001DEC10F0E8B013D02EC0D9FF2DC0DAFFC6
:102B0000165017B81E5017B661EC12F017A64BEC12
:102B100012F0E82C04D0050EEBEC11F04DD7252A6D
:102B2000050E25180FE101902A66249E230E01163A
:102B3000006A3338030B306E74EC10F0040EB5EC01
:102B400012F019D0050EEBEC11F043D701A008D01C
:102B5000252A030E256004D0040EEBEC11F052D6AA
:102B60002A66249E0190230E0116006A3338030B57
:102B7000306E74EC10F0256A010E17B004D001B06D
:102B80000BD035A209D0130E306E110E2FEC10F0C1
:102B9000050E24B0FF0E2490EBEC11F037BA02D0F2
:102BA00037AC0400040EC1EC12F001A0006A005022
:102BB000D8B40190230E01A00116020E306E260E2D
:102BC0002FEC10F0010E306E290E2FEC10F00A0ED3
:102BD000306E2A0E2FEC10F0000E306E2B0E2FEC04
:102BE00010F035501F0B07E017B005D05B0E306EAC
:102BF000110E2FEC10F0306A0050351403E1230E53
:102C000001160190010E01A0100E35A2010EEBEC91
:102C100011F017A000D0090EF46EF32EFED7F42E9B
:102C2000FCD7809496EF1BF00190230E0116006AEA
:102C3000A2D71200010EDC520BE1DC5209E608E0DB
:102C4000DFCFE3FFDF44080F02E2F80F1200010EAE
:102C5000E368120095EC19F003E1400E48EC19F01E
:102C600055C057F053C055F054C056F052C054F000
:102C7000305062EC19F030501200D9EC19F09D98E8
:102C8000AC9A5194519E51962C0E586E920E596EDC
:102C900012009E989EAA1200130EC2EC19F02AECA4
:102CA00016F051A206D0100AE87803E1536A9DEFAE
:102CB00023F03F943F82518602E1518E07D0F80AFB
:102CC00002E1F80A03D0F80A31625196FDEC19F0DE
:102CD0001DEC19F0130EC2EC19F02D0E586E0C0EEF
:102CE000596E9EAA12002AEC16F0FCEC18F09EBA5F
:102CF000FAD711EC1AF0E86601D01200080ECCECFD
:102D000019F0300E586E720E596E1200F2A4E2D70E
:102D1000D59EF29AF294306A5AC0DAFF5B50D96EAF
:102D2000FE0BD8B41ED1DD5051B41FD145B20AD02C
:102D3000566203D0DF5057180EE051A245B002D0C2
:102D400045900FD1DC500D0AFBE1DD50DF500A0A3F
:102D5000F7E1452A45B24590308051BE02D051B6C8
:102D60003086305048EC19F051A20FD03F50700B14
:102D70000BE0100A09E0300A07E0600A05E0300ABB
:102D800004E13F9C3F9A3F88519251A676D75AC0A2
:102D9000DAFFD96A030EDC6201D07ED051A804D0DC
:102DA00051965198519A69D7DFA69FD0080EDF62DD
:102DB00026D0DC6614D0DC5003E1ACEC18F088D0EF
:102DC000DF4C15D00A0EDF5C12E009E3F90F02E2D6
:102DD000060F1BD004E0E82C02D0060E16D0010E20
:102DE000D96AD982DF6E030EADEC18F071D0DC6ABF
:102DF000DC6AACEC18F0FF0E56EC19F069D00B0E43
:102E0000DF622ED0DC6ADC6A070EE844E828E2CFF5
:102E100056F0E1CF57F013EED0F0E3CFDCFFE8043B
:102E2000E3CFDCFF56C0E2FF57C0E1FFACEC18F087
:102E30004FD001000003000E54656C656D65636141
:102E40006E6971756520010E4F7369747261636BF1
:102E5000205847432D53020676312E353320FF305C
:102E60002B0EDE62BCD70E0EDF62B9D7FC0EDC146F
:102E7000030ED8A4B5D7DF6601D0B2D7F86A320EF8
:102E8000F66E2E0EF76E0900F550DC6EFCE70900B9
:102E9000F550ADEC18F01CD0E2CF56F0E1CF57F072
:102EA000030EBEEC18F0C10EE76E2DEC19F05B506E
:102EB000070AD8A494D71AEC16F056C0E2FF57C000
:102EC000E1FFD906D906D906DF6E030FD96ADF6E96
:102ED000D59EF29AF294F80ED76ED66AD58EF28A03
:102EE0002F0E586ED20E596E1200100EDF621CD0DB
:102EF000E2CF56F0E1CF57F0070EBEEC18F0C00E4F
:102F0000E76E2DEC19F01AEC16F0050ED96EDE44C2
:102F1000DF6265D75B50F80FDF6261D756C0E2FF12
:102F200057C0E1FF060ED2D7060EDF6258D7E2CFB8
:102F300056F0E1CF57F0060EBEEC18F0C00EE76E6B
:102F40002DEC19F0DC50DCCF30F0DC6E30C0DCFF53
:102F5000010EE36AE38056C0E2FF57C0E1FF060EB0
:102F6000B5D73082305048EC19F051A23DEF16F041
:102F700051985196080E5B6213D0D96E5AC0DAFF91
:102F8000040EDD620DD07D0EDD620AD00F0EA96E3B
:102F9000FE0EF29EB1EC0BF0020E21EC02F0FF00EF
:102FA0003FBAD8EF17F03FBCD8EF17F03FA80DD0CD
:102FB00023EED2F0FE0E51B0F00EDF24D8B005D0D3
:102FC0003FBA8CEF23F03DEF16F0010EF46EF36E76
:102FD000FF009EAA03D0526853685BD6080ECCEC63
:102FE00019F0EEEC18F0E8A01200ACA21200D59E89
:102FF000F29AF2949D9A828A82885B6A566A0E0ED1
:10300000DBB856880D0EDBB4568ADB505BC0D9FFA7
:103010005AC0DAFF0CE05684DC8EDC6ED906AB0EAB
:10302000DE18030ED8B4DF6E56B81ED007D00B0ED4
:10303000DC62568ED906DF5056B817D0506E5C5001
:10304000306E5368526862EC19F09D889D9A9E9A82
:1030500086EC19F0565048EC19F0300E586ED20E2E
:10306000596E9EB836D012005698565048EC19F05A
:1030700004D6D59EF29AF294828850065BC0D9FF9E
:103080005AC0DAFFDC50306E62EC19F086EC19F0B1
:103090005B2A5E045D245B1803E09EB8EED7120045
:1030A000040ECCEC19F0300E586EB20E596E9D988D
:1030B0001200F2A41200ACB204D0020ECCEC19F053
:1030C0001200504E1CD082989D98DCEC19F0000044
:1030D000D4D551BAD2D7504E12D05BC0D9FF5AC006
:1030E000DAFFDC50306E62EC19F086EC19F05B2AE6
:1030F0009EB8EFD7300E586ED20E596E1200535054
:1031000045A045B20A0E306E86EC19F0310E586EAD
:103110001A0E596E9EB801D01200525045A045B209
:103120000D0E306E86EC19F0080ECCEC19F0310E55
:10313000586E3A0E596E9D981200F2A41200ACB26D
:103140009CD5080ECCEC19F0120005005850FE6E0C
:103150005950FD6EFF6A1200060ED96ADF6EE80450
:10316000E2CF56F0E1CF57F0BEEC18F00F0EE36A55
:10317000E38456C0E2FF57C0E1FF1200506E11EE2B
:1031800020F00F0EE126000EE222DAB0100EE1264A
:10319000000EE222200EDAB0100F406E020EE76E33
:1031A000F00EE1160A0EDACFE3FF0B0E50C0E3FF7C
:1031B000090E5CC0E3FF501C030F506A3FB250364B
:1031C0000D0E50C0E3FF0E0EE36A51BEE38851B806
:1031D000E38EE38C0C0EE36AE384120040C0D9FF57
:1031E000010EDA6E0F0EDBA4000C51A8010C5E6616
:1031F000000C5198518A020C5B2A03E151845B0652
:1032000012005AC0DAFF5BC0D9FFDF6EDACF5AF086
:10321000D9CF5BF012009E98F2A40CD0D59EF29A02
:10322000F294060051A205D02C0E586EB20E596EC3
:10323000120012009EAA06001200040E5A6406D064
:1032400051BA06D05A6E000E5B6E120051BAFAD710
:10325000050E5A6E000E5B6E1200020EDCCFE3FF0D
:10326000030EDCCFE3FF1200030EDCCFE3FF020E00
:10327000DCCFE3FF120023EED0F0D926D926DE2AD8
:10328000D8A01200DF2ADFAE1200DD06DF06120032
:1032900023EECFF003D0DE2A02E3DF2AD890DE52FD
:1032A000E830F9E2DE02DE02FBE1120023EED0F0AC
:1032B00002D0DE6ADE6AD890E830FBE2DE02DE028F
:1032C000FBE11200531A53385318F46EE840F41817
:1032D000E830E8B2D8705330F46E536A5332F430A9
:1032E000F41A5330531AF4BE53805250531AF4CF89
:1032F00052F012003F9030383018E8B03F70E8B21A
:103300003F70E8B43F70E8B63F701200AC8AAC90F2
:103310003FB807D07AEC19F03FAC3F703FAA3FBCF2
:103320003FB0AC7030C0ADFF1200AB30E8B0AB982E
:10333000AB88AECF30F0ABAC1DD0F36E7AEC19F0A9
:103340003F34E804030B020FE870E83851B204D0B0
:103350003F1401E1518412008F093F16700E3F1493
:10336000F3B202D0F8E101D0AB7C100EABBC700E12
:103370003F121200D894E8A2120051B2F5D7D884B7
:1033800051841200D59EF29AF2943902F450F80B4F
:10339000080ED8B4F46E04D0D59EF29AF294390295
:1033A000F41CD76EF31CD66ED650D750D58EF28A49
:1033B0001200829852685368D59EF29AF294829ACB
:1033C000AC98AB8E51B205D0AB9C3FBAAB8C3FBC36
:1033D000AB8C9D8AAB889EAA0AD0AB50AE509EAAF9
:1033E00006D0AB50AE509EAA02D0AB50AE50AB5000
:1033F000060B02E0AB98AB881200519A5C6E12008B
:103400000F0B316402D0519812005C380F0BE804A6
:10341000FAE63164F8D751B8518A517851B85186DB
:103420001200000C51AA000C5E04FF0F5B64000C3C
:103430005DC050F05C500F0B3162508E502A9D8859
:103440009D9A9E9A828A010C824B3F01353F730000
:10345000838B005266000107840408FEFF0035A23A
:10346000CFEF21F000B203D001B0CFEF21F0480E32
:10347000F66E340EF76EB9EC11F0306A74EC10F0A1
:103480002A6A010EEBEC11F041EC10F0200E01B0B5
:10349000E10E836E82968286000E836E829682860D
:1034A0008296828682968286000E01B0010E836E1D
:1034B00082968286000E836E829682860C0E306E15
:1034C000D88052EC11F02688280EEBEC11F030BABF
:1034D000EED05E0E01B0000E306E250E2FEC10F017
:1034E000070EEBEC11F0030E1DEC10F0700A700BE0
:1034F000E866DDD0280EEAEC11F030BAD8D00A0E1A
:103500001DEC10F03F0BE866D2D093EC12F0256A68
:10351000400E1B6E1A6A300E196E040E186E166E6F
:1035200017BC178E008201B010D00180306A74EC95
:1035300010F06BEC1BF026880A0EEBEC11F030BAA1
:10354000B6D0306A250E2FEC10F0E1EC12F0E82C2A
:10355000BCD01C68256A010EEBEC11F0EFEC12F008
:10356000E8BE09D0B5EC12F03066AFD0020EEBEC3D
:1035700011F00400EAD717B63BD041EC10F0600E12
:10358000836E82968286080E236E7D0E226E2EC07A
:10359000D9FF2DC0DAFF040E44EC12F02C508FEC52
:1035A00011F0231E221E080E306ED88049EC11F057
:1035B00026842688640EEBEC11F030BA69D05E0EDA
:1035C000306E250E2FEC10F0400EEAEC11F030BA00
:1035D0005FD00A0E1DEC10F03F0B01E059D0040E35
:1035E0001DEC10F000006BEC1BF0800EEBEC11F00A
:1035F000306A250E2FEC10F041EC10F0E10E836ED6
:1036000082968286836A8296828682968286829655
:103610008286AB0E236EB70E226E1F048FEC11F064
:103620002C508FEC11F0231E221E080E306ED88015
:1036300049EC11F02688460EEBEC11F030BA28D098
:103640000B0EEBEC11F0030E1DEC10F0700B700A7A
:10365000E8661ED0D50EEAEC11F030BA19D00A0E89
:103660001DEC10F03F0B01E013D02EC0D9FF2DC090
:10367000DAFF165017B81E5017B661EC12F017A6F5
:103680004BEC12F0E82C04D0050EEBEC11F066D7F1
:10369000252A040E256407D0040EB5EC12F0040EA2
:1036A000EBEC11F0F1D6050EEBEC11F064D701A0B4
:1036B00005D0252A020E2564F2D724800190006AE5
:1036C000230E0116306A74EC10F0256A010EEBEC43
:1036D00011F0CFEF21F0010E306E090E2FEC10F03B
:1036E000956A810E836E846A829682868480836E58
:1036F00082968286846A800E836E82968286848217
:10370000956A20EE05F0DF1C306E6CEC11F0836ED4
:10371000829682861200825B3F3F19133F008373BB
:1037200008A9881E010784060363630035A46FEFB0
:1037300020F000B403D001B06FEF20F0160EF66E4B
:10374000370EF76EB9EC11F0050E01B03F0E306E7A
:103750008DEC10F02A6A279427961C68256A24822B
:103760002494010EEBEC11F0000E4F6E61EC10F0A2
:1037700041EC10F0520E836E8296828600D0090EC4
:10378000F46EF32EFED7F42EFCD78094070E306E25
:103790000F0E2FEC10F0020E306ED88052EC11F0AC
:1037A0002688020EEBEC11F030BACAD3306A0F0E45
:1037B0002FEC10F0050EEAEC11F02F2A30BA01D0F0
:1037C00007D04F2A020E4F62D1D7000E4F6EB8D3EA
:1037D0000A0E1DEC10F0370BE866B2D3020E1DEC9A
:1037E00010F0306E400F286ED8B0AAD31F0BE8300F
:1037F00007E2E83005E2E83003E2E83001E2010ADE
:10380000E8669ED3FC0E271628462846030E281687
:10381000020E1DEC10F028A207D0FE0BE8660198FE
:103820001A6AE8B2018E00D0030EEBEC11F041EC05
:1038300010F02734060B930F836E829682862A50EF
:10384000070B306E2A50280BE8443010200F836E8F
:103850008296828620EE04F027500C0BD9262A503F
:103860000EE0DECF83FF82968286F80FE866F9E7E6
:10387000070B306EE83830120F0E2FEC10F0030EED
:10388000306ED88052EC11F026880A0EEBEC11F065
:1038900030BA56D3080EEAEC11F030BA51D320EE0C
:1038A00004F02744E8440C0BD9262A38E844070BD7
:1038B000D92627500C0BE866D926D9CF23F0070E5E
:1038C0002AB47F0ED8902AA2E830D8902AA2E830F5
:1038D000D8902AA0E830DF14226E0A0E1DEC10F0FA
:1038E000E830040E01E3000EBFEC1FF023C0D9FF47
:1038F0002250DF12F31A24AC06D0249C360AF00BB7
:103900000FE1358A0DD024AA06D0249A160AF00BAE
:1039100007E1248C05D024A803D0000A01E1248A01
:10392000DF500F0B216E0A0E1DEC10F0370B0BE071
:10393000340BE86605D30B0E1DEC10F02A6E020E58
:10394000EBEC11F074D7F366FBD2020EEBEC11F046
:1039500041EC10F02734060B930F836E829682861B
:10396000700E836E8296828620EE04F02744E8442F
:103970000C0BD926000EDA2227500C0BE866D9264C
:10398000040E20EC12F0836E829682860F0E306E4B
:10399000D88052EC11F026880B0EEBEC11F030BA07
:1039A000CFD2080EEAEC11F030BACAD20A0E1DECE2
:1039B00010F03F0BE866C4D2272A2750030B286279
:1039C00033D7020E1DEC10F0E8B4BAD2080AD8B40E
:1039D00000EF1DF0200AD8B400EF1DF0300AD8B473
:1039E0000AEF1DF0200AD8B40AEF1DF0180AD8B467
:1039F0001FEF1DF0200AD8B413EF1DF029EF1DF0C2
:103A0000018C0198100E166E196E186E1B6A040E4A
:103A10001A6E1FD0018C0198100E166E186E1B6A5C
:103A2000100E1A6E16D0019C0188400E1B6E000EFF
:103A30001A6E100E196E040E186E166E0AD0019CC6
:103A40000198018E100E166E196E186E1B6A040E08
:103A50001A6E0180E1CF23F0E2CF22F027500C0B49
:103A600020EE04F0D926DF50E840E8400C0BE16E70
:103A70002AB402D035AA04D01AA802D00C0A23E135
:103A8000020EE26EDE50E762178EE66EDE50E762EF
:103A9000178EE66EDE50E762178EE66EDE50E76246
:103AA000178EE66E17AE0FD02A6609D0E198E76A46
:103AB000040EE126E198E76AE126E198E76A086AE0
:103AC000096A0A6A0B6A23C0E1FF22C0E2FF008490
:103AD000020E286201D019D000C0E0F101C0E1F16E
:103AE00002C0E2F103C0E3F104C0E6F105C0E7F172
:103AF00006C0E4F107C0E5F108C0E8F109C0E9F14A
:103B00000AC0EAF10BC0EBF118D000C0E0F101C02F
:103B1000E1F102C0E2F103C0E3F105C0EBF106C040
:103B2000E8F107C0E9F108C0E6F109C0E7F10AC011
:103B3000E4F10BC0E5F10CC0EAF13F0E306E8DEC04
:103B400010F0E1EC12F0E82CE2D17F0E146E01AE21
:103B500032D0020EEBEC11F0030EEBEC11F0CBD1F6
:103B600041EC10F0E00E836E82968286500E836EDA
:103B7000829682860F0E306ED88052EC11F01B0EAA
:103B8000EAEC11F030BAAFD10A0E1DEC10F03F0B89
:103B900001E0A9D1010EEBEC11F041EC10F00A0E9E
:103BA000836E82968286000E836E82968286280EAF
:103BB000EBEC11F098D1020EEBEC11F024B411D023
:103BC00001AC07D0100E1A6204D02A661B683F0EA3
:103BD0001A6EEFEC12F02484E8BE03D0B5EC12F0BC
:103BE00096D101AC50D035BE02D024A604D024A278
:103BF0004AD0249224D001A205D02C50F00B02E12F
:103C00002B50F5E024A237D024922B0E2BB2810E3C
:103C10002BB02B0F2C2403E2D50F2C6E05D02C6E6D
:103C20002B2A020E2BB4DAD7CE0E2C24F66E3F0EC2
:103C3000D8B0010FF76EF86A0800F5502C6E2B66AD
:103C400004D035AA20D01AA81ED0040E2AA4C6D7A4
:103C5000060E2A6E279427962BB227862BB0278430
:103C600020EE04F027500C0BD926E844E844300A33
:103C70002118DF6E26D1F00E2CAEFC0E2C10E82899
:103C8000000E2C22CCE001B883D02CBE04D02C3006
:103C9000E8301F0B03D02C38070B2009146204D026
:103CA0007F0AD8A475D07F0A146E41EC10F015502D
:103CB000836E82968286000E836E82968286020EC4
:103CC000306E220E2FEC10F00B0E306E010E2FEC2A
:103CD00010F0040EEBEC11F000000A0E1DEC10F0D9
:103CE000E8BCE2D0010E1DEC10F0000041EC10F039
:103CF000600E15B4610E836E829682862C50836EA0
:103D00008296828620EE04F027500C0BD926040EF2
:103D100020EC12F0040E1DEC10F00000070E306EC7
:103D2000220E2FEC10F00C0E306E010E2FEC10F066
:103D30002684200EEBEC11F030BAB6D00A0E1DEC42
:103D400010F07F0B01E0B0D0050E1DEC10F0070B5A
:103D5000D8A4AAD0040EEBEC11F041EC10F0030E45
:103D6000306E220E2FEC10F0140E306E010E2FEC80
:103D700010F02684400EEBEC11F0090E1DEC10F053
:103D8000E8A692D00A0E1DEC10F07F0B01E08CD05B
:103D900017B662D041EC10F0A20E01A8A00E836EFF
:103DA000829682862C50836E829682862EC0D9FFA0
:103DB0002DC0DAFF1650306E01B820EC12F00F0E55
:103DC000306ED88052EC11F0780EEAEC11F001B8A8
:103DD00033D030BA69D00A0E1DEC10F0370B01E079
:103DE00082D0020E1DEC10F00A0AD8A47CD0040E7A
:103DF000EBEC11F041EC10F02EC0D9FF2DC0DAFF32
:103E00001650306E20EC12F00F0E306ED88052EC4F
:103E100011F0780EEAEC11F030BA65D00A0E1DEC04
:103E200010F0370B01E05FD0020E1DEC10F00A0A13
:103E3000D8A459D02494BFD630BA36D00A0E1DEC7F
:103E400010F0370B01E030D0020E1DEC10F00A0A22
:103E5000D8A42AD02494AFD641EC10F0300E836E53
:103E6000829682862C50836E829682860F0E306EEA
:103E7000D88052EC11F0500EEAEC11F030BA14D0A8
:103E8000040E1DEC10F0E84C0FD00A0E1DEC10F0E3
:103E90003F0B01E009D02EC0D9FF2DC0DAFF1E5024
:103EA00061EC12F0249487D601B81DD0252A050EA6
:103EB00025601DD061EC10F00C0E1526800E15BA91
:103EC000156E41EC10F0500E836E82968286836AE6
:103ED00082968286070E306ED88052EC11F0280E42
:103EE000EAEC11F043D4252A040E256425D061ECB8
:103EF00010F07F0E146E0190006A230E0116050E5D
:103F0000306E8DEC10F00094040EB5EC12F0040E3F
:103F1000EBEC11F041EC10F0500E836E829682862D
:103F2000836A82968286070E306ED88052EC11F03A
:103F3000280EEAEC11F016D0050EEBEC11F028D7A4
:103F400001A008D0252A030E256004D0040EEBEC56
:103F500011F00CD40190006A230E0116050E306E8C
:103F60008DEC10F0090E1DEC10F0F70B306E090E01
:103F70002FEC10F0256A010EEBEC11F0B0D0306E92
:103F8000179C956A800E836E846A82968286020EE2
:103F90008D6E9568F36A305010E082920000835075
:103FA0008282F31ADF62178CDE6E302EF6D7829291
:103FB000000083508282F31A1200C00EDF16829234
:103FC0000000835082823F0BDF12F31A12000405B7
:103FD0000608090A0C0D0E10111214151618191ADC
:103FE0001C1D1E20212224252628292A2C2D2E3076
:103FF000313234353638393A3C3D3E404142444511
:104000004648494A4C4D4E50515254555658595AAB
:104010005C5D5E60616264656668696A6C6D6E7045
:10402000717274757678797A7C7D7E8081828384E2
:1040300085868788898A8B8C8D8E909192939495B2
:10404000969798999A9B9C9D9EA0A1A2A3A4A5A691
:10405000A7A8A9AAABACADAEB0B1B2B3B4B5B6B770
:10406000B8B9BABBBCBDBEC0C1C2C3C4C5C6C7C84F
:10407000C9CACBCCCDCED0D1D2D3D4D5D6D7D8D92E
:10408000DADBDCDDDEE0E1E2E3E4E5E6E7E8E9EA0D
:10409000EBECEDEEF0F1F2F3F4F5F6F7F8F9FAFBEC
:1040A000FCFDFE0000000000000000000000000019
:1040B0000000000000000000000000000000000000
:1040C0000000000000000000824B3F0620133F006C
:1040D000837319A988FE010084282CFFFF0035A6F0
:1040E0002FEF1AF000B603D001B02FEF1AF0C80E70
:1040F000F66E400EF76EB9EC11F0020E306E74ECF5
:1041000010F02A6A010EEBEC11F041EC10F0010EF8
:10411000836E829682860B0E836E829682863F0E17
:10412000836E82968286800E836E829682862C0EA5
:10413000306ED88052EC11F02688150EEBEC11F0A1
:1041400030BAF2D0150EEAEC11F0030E1DEC10F0AF
:10415000700B700AE86601D005D0132A030E1362B3
:10416000D4D75BD0136A1F0EEAEC11F030BADCD062
:104170000A0E1DEC10F03F0BE866D6D0040E1DECC5
:1041800010F00C6E1B0AD8A4CFD021EEC0F00CC0EA
:10419000E8FF61EC12F00E0EEBEC11F001EEE4F032
:1041A000C2C1E8FFEE620DD0C3C1E8FFEE6209D0E4
:1041B000C4C1E8FFEE6205D0C5C1E8FFEE6201D0E0
:1041C00017D0178EC2C104F0C3C105F0C4C106F0F8
:1041D000C5C107F004C0E4F105C0E5F106C0E6F191
:1041E00007C0E7F101EEE8F0EE6AEE6AEE6AEE6A09
:1041F00001800192006A0086018C040E196E186E0F
:10420000020E306E74EC10F00400256B120EEBEC15
:1042100011F001B07AD72FEF1AF041EC10F0050E33
:10422000836E82968286000E836E82968286000E50
:10423000836E829682862C0E306ED88052EC11F0FE
:104240002688150EEBEC11F030BA64D0070EEAECBC
:1042500011F0030E1DEC10F0700B700AE8665AD0D6
:104260001F0EEAEC11F030BA55D00A0E1DEC10F01A
:104270003F0BE86655D0040E1DEC10F00C6E0C0AD6
:10428000D8A44ED021EEC0F00CC0E8FF61EC12F0D3
:104290000E0EEBEC11F001EEE4F0C3C1E8FFEE62AC
:1042A0000DD0C4C1E8FFEE6209D0C1C1E8FFEE62E3
:1042B00005D0C2C1E8FFEE6201D017D0178EC1C190
:1042C00004F0C2C105F0C3C106F0C4C107F0C3C108
:1042D000E4F1C4C1E5F1C1C1E6F1C2C1E7F101EE0B
:1042E000E8F0EE6AEE6AEE6AEE6A01800192006A18
:1042F0000086018C040E196E186E020E306E74EC7E
:1043000010F00400256B120EEBEC11F001B085D714
:104310002FEF1AF001A012D0252A0A0E25600ED028
:10432000040EEBEC11F079D701A008D0252A030E7A
:10433000256004D0040EEBEC11F0E7D60190006A82
:10434000230E0116020E306E74EC10F0256A010E79
:10435000EBEC11F000D0090EF46EF32EFED7F42E24
:10436000FCD780942FEF1AF0C20E836E829682865D
:104370002C0E306ED8801200E20E836E82968286FA
:104380002C0E306ED8801200825B3F002F3F3F0022
:10439000838B14D068E0010084080812E00035A87F
:1043A000ECEF13F000B803D001B0ECEF13F0880E7F
:1043B000F66E430EF76EB9EC11F0010E306E74EC30
:1043C00010F02A6A010EEBEC11F001B03BD041EC89
:1043D00010F00A0E836E82968286200E306ED89080
:1043E00052EC11F0200EEBEC11F0040E1DEC10F06D
:1043F000000041EC10F00C0E836E82968286080E4F
:10440000306ED88052EC11F00C0EEBEC11F0030E74
:104410001DEC10F0700A700BE86632D1300EEAEC39
:1044200011F030BA2DD10A0E1DEC10F000003F0B38
:10443000E86626D1080E20EE0CF0A0EC12F0050E76
:10444000EBEC11F041EC10F0810E836E82968286C7
:1044500020EE0CF001B020EE04F0080E20EC12F07B
:10446000080E306ED88052EC11F0600EEAEC11F0BC
:1044700030BA06D10A0E1DEC10F03F0BE86600D1F1
:104480009DEC12F01B6A010E1A6E080E196E186E62
:10449000166E018017BC178E008820EE08F0DFB67C
:1044A00002D0100E1A6E010E306E74EC10F005C0C2
:1044B000E4F104C0E5F107C0E6F106C0E7F109C088
:1044C000E8F108C0E9F10BC0EAF10AC0EBF1E1EC58
:1044D00012F0E82CE8D01C68256A050EEBEC11F010
:1044E000EFEC12F0E8BE09D0B5EC12F03066DBD08C
:1044F000020EEBEC11F00400DAD72B5014183BE05D
:10450000240E306E130EA8EC11F041EC10F0840E66
:10451000836E829682862B50E838836E82968286DE
:10452000040E306ED88052EC11F0500EEAEC11F00F
:1045300030C0D9FFE00E306E120EA8EC11F0D9BADF
:104540008AD00A0E1DEC10F0370BE86684D0080EF6
:1045500020EE0CF0A0EC12F020EE11F0DFBA06D045
:104560002B5004E0020EB5EC12F09DD02BC014F0DD
:10457000050EEBEC11F017B63ED0240E306E100E87
:10458000A8EC11F041EC10F0870E836E82968286C3
:104590002C50836E829682862EC0D9FF2DC0DAFF02
:1045A000080E20EC12F0040E306ED88052EC11F0A0
:1045B000FF0EEAEC11F0D96EE00E306E120EA8EC90
:1045C00011F0D9BA12D00A0E1DEC10F03F0B0DE11C
:1045D0002EC0D9FF2DC0DAFF1E504BEC12F0E82C94
:1045E00004D0050EEBEC11F07BD70C0E1DEC10F097
:1045F0000109EBEC11F041EC10F00C0E836E829689
:104600008286E00E226E120E236E2C508FEC11F07B
:10461000231E221E080E306ED88049EC11F0600E69
:10462000EAEC11F030BA17D00A0E1DEC10F03F0B77
:1046300001E011D02EC0D9FF2DC0DAFF1E5017B6F1
:1046400061EC12F017A64BEC12F0E82C04D0050E2A
:10465000EBEC11F045D7252A050E25180DE1019048
:10466000006A230E0116146A010E306E74EC10F00D
:10467000040EB5EC12F017D0050EEBEC11F03DD79F
:1046800001A008D0252A030E256004D0050EEBEC0E
:1046900011F09DD60190006A230E0116146A010ED6
:1046A000306E74EC10F0256A010EEBEC11F0ECEFBB
:1046B00013F021EE20F00F0EDB6605D0040E5A6ECB
:1046C000000E5B6E1200100FDB6605D0050E5A6EF1
:1046D000000E5B6E1200DB6A21EE20F00F0EDB6A2B
:1046E000EDD795EC19F030505326100AE87806E122
:1046F00052A0060052A0502A52701200529012008E
:10470000010ED96E020EDF66050FD96EFD0EDF6E4B
:10471000D950D96ADF6E1200D9EC19F09D98AC9A85
:10472000470E586E2A0E596E12009E989EAA1200CD
:10473000180ECCEC19F095EC19F03F923F8451948F
:10474000519E5196519C30505290100A17E051A240
:10475000E7D751965198140A05E123EED2F051B2F1
:10476000DF6ADED72C0E586E920E596E30505268AA
:10477000536862EC19F0305059EF16F0470E586E3E
:10478000860E596E1200100E536E0BEC19F0180EB7
:10479000CCEC19F071EC23F0050A07E0070A0EE0F3
:1047A000470E586E2A0E596E120023EED2F051B207
:1047B000DF6A470E586EC60E596E1200480E586ECC
:1047C000360E596E12000BEC19F095EC19F03050C2
:1047D0003162A2D7311808E1180ECCEC19F0470E5F
:1047E000586EF00E596E1200D59EF29AF29494D73C
:1047F0009E989EBA95D7F2A41200D59EF29AF29492
:104800009D9A828A82889D889D9A9E9A5B6A5BC0E7
:10481000D9FF5AC0DAFFEEEC18F0E8A009D0100E6C
:10482000306E86EC19F04C0E586EE60E596E120082
:10483000040E4FEF26F00BEC19F0180ECCEC19F02B
:1048400095EC19F030505326406605D05186FF0A8A
:1048500007E1518E08D0518C51963162519C05D0A0
:10486000FF0A3162519651B6406A59EC23F0480E66
:10487000586E780E596E12000BEC19F0180ECCEC35
:1048800019F071EC23F0506E502A480E586E940EB9
:10489000596E12000BEC19F0180ECCEC19F071ECFB
:1048A00023F05006FCEC18F0000A05E1480E586EA3
:1048B000E40E596E1200480E586EC00E596E12006A
:1048C0000BEC19F0180ECCEC19F0500671EC23F03B
:1048D000FCEC18F0060E5B621200480E586EE40EF7
:1048E000596E12000BEC19F0180ECCEC19F071ECAB
:1048F00023F05006FCEC18F0490E586E020E596E6B
:1049000012000BEC19F0400ECCEC19F0504E05D013
:1049100071EC23F0FCEC18F0120095EC19F0FCECB3
:1049200018F03050D9CF50F05362D1D151B4CFD11B
:1049300051BC98D151B605D0D59EF29AF2945192BD
:10494000EBD6556AE2CF56F0E1CF57F011EE20F0EA
:104950000F0EE36A020EE38E030EE38E0D0EE36A82
:104960000E0EE39011EE30F0E390020EE38E030E94
:10497000E38E0D0EE36A0F0EE36A56C0E2FF57C0E6
:10498000E1FF010ED96EDF66060EE828D96E010F31
:104990005018D8B45ED10F0EDF6243D03F0EDE6EEA
:1049A000240EDE6E010EDE6EF86A590EF66E2E0EC5
:1049B000F76E0900F550E8BC090FE838F00B306ECF
:1049C00009000900F550E8BC090F0F0B3010DE6E2E
:1049D0000B0EDE6E510EF66E2E0EF76E0900F550C0
:1049E000DE6E0900F550DE6E0900F550DE6E09003E
:1049F000F550DE6E0900F550DE6E090009002D0E3F
:104A0000DE6E0900F550DE6E0900F550DE6E09001D
:104A1000F550DE6E0900F550DE6E0900F550DE6ED1
:104A20001ED1FA0EDF620ED0DE2AD92850BE11D177
:104A3000505E210E50600DD1D92ADD50DE6E502E11
:104A4000FBD70DD1300EDF620FD0600EDE6E800E10
:104A5000DE6E000EDE6E010EDE6E100EDE6E000EDD
:104A6000DE6E000EDE6EFBD0310EDF6209D0610E0D
:104A7000DE6E010E01A0000EDE6E010EDE6EEFD0C6
:104A8000A20EDF6213D0D20EDE6E000EE2CF56F021
:104A9000E1CF57F013EED0F0E3CFDEFFE828E8A631
:104AA000FBD756C0E2FF57C0E1FFD9D0A40EDF62AA
:104AB00018D0FE0EDE6ED950D96ADF6E306E000E51
:104AC000E2CF56F0E1CF57F013EED0F0E66AE828D7
:104AD000E8A6FCD756C0E2FF57C0E1FF30C0D9FFBF
:104AE000BED0330EDF6205D0630EDE6E000EDE6ECA
:104AF000B6D0360EDF6237D0300FDE6ED92AE2CF65
:104B000056F0E1CF57F0D950BEEC18F0D906020E9E
:104B1000DB50DE6E03E10E0EE38004D0FE0B060ACE
:104B2000E86693D0C10EE76EDE50680A03E0690ABA
:104B300001E08BD034EC19F0DC50D8B486D0790E7B
:104B4000DF6083D0DC6681D0010EE126D906DF501C
:104B5000E76EE844D924FB0FD96ADF6E56C0E2FF46
:104B600057C0E1FF7FD0040EDF6218D0300FDE6E39
:104B7000E2CF56F0E1CF57F0D950BEEC18F0C10E9D
:104B8000E76E34EC19F0010EE36AE380D904D96AC8
:104B9000DF6E56C0E2FF57C0E1FF64D0370EDF6220
:104BA00035D0FE0EDE6ED92AE2CF56F0E1CF57F0B7
:104BB000D950060FBEEC18F0010EDB5003E10E0ECB
:104BC000E38004D0FE0B060AE8663FD0C00EE76E15
:104BD000DE50680A03E0690A01E037D034EC19F0CE
:104BE000DC50D8B432D0790EDF602FD0DC662DD007
:104BF000010EE126D906DF50E76ED950FA0FD96AC7
:104C0000DF6E56C0E2FF57C0E1FF2CD0140EDF620A
:104C100020D0FE0EDE6ED92AE2CF56F0E1CF57F05B
:104C2000D950020FBEEC18F0C00EE76ED90634EC76
:104C300019F0010EE36AE380D950FD0FD96ADF6EE7
:104C400056C0E2FF57C0E1FF0DD056C0E2FF57C08B
:104C5000E1FF80EC23F0020EB0EC18F003D0D90491
:104C6000ADEC18F0519251BE57D54C0E586E740EE3
:104C7000596E12009E989EBA53D5F2A41200D59E8A
:104C8000F29AF2949D9A828A82889D889D9A9E9A31
:104C9000060E51AC04D0020E3BEC19F0150E306E2E
:104CA00086EC19F0080ECCEC19F09D984C0E586E5D
:104CB000B60E596E1200F2A41200ACB204D0080E67
:104CC000CCEC19F012009D98AC9A8CEF23F0D59E95
:104CD000F29AF294030E3BEC19F051A21DD55196B5
:104CE00051983DEF16F0120E536E020E306E86ECA8
:104CF00019F052904C0E586EFE0E596E1200315043
:104D00005326306E86EC19F04D0E586E120E596E09
:104D1000120040C0D9FF010EDA6E0D0EDBCF30F06D
:104D20000A0EDB50DA6E5A6ED96A5B6A306680EC26
:104D300023F0DE505326306E506E86EC19F0305062
:104D4000100A03E1527052B0120052904D0E586E8C
:104D5000560E596E12005BC0D9FF5AC0DAFFDC5004
:104D60005326306E86EC19F03050100A03E1527071
:104D700052B01200D9CF5BF0DACF5AF05290502ED9
:104D800012004D0E586E8C0E596E12005350306E3C
:104D900086EC19F0080ECCEC19F04D0E586EA60EEC
:104DA000596E9D981200F2A41200ACB204D0080E05
:104DB000CCEC19F01200D9EC19F09D98AC9A4D0E7C
:104DC000586EC80E596E12009E989EAA1200180EB8
:104DD000CCEC19F095EC19F030505290060E306280
:104DE00009D040C0D9FF010EDA6E0F0EDB6A406AAF
:104DF0008CEF23F0150E3018E866010E3BEC19F02D
:104E0000E8A004D0552A55B09DEF23F0556A40C064
:104E1000D9FF010EDA6E0F0EDB6A406A9DEF23F0B8
:020000040030CA
:02000000FFFA05
:02000200F6FE08
:020006007BFF7E
:02000800F0BF47
:02000A00FFBF36
:02000C00FFBF34
:00000001FF
